BL51 BANKED LINKER/LOCATER V6.22                                                        05/19/2022  17:58:17  PAGE 1


BL51 BANKED LINKER/LOCATER V6.22, INVOKED BY:
C:\KEIL_V5\C51\BIN\BL51.EXE .\Objects\OPTIONS_SN8F5835.obj, .\Objects\main.obj, .\Objects\uart.obj TO .\Objects\SN8F5835
>> _Test Code PRINT (.\Listings\SN8F5835_Test Code.m51) RAMSIZE (256)


MEMORY MODEL: SMALL


INPUT MODULES INCLUDED:
  .\Objects\OPTIONS_SN8F5835.obj (OPTIONS_SN8F5835)
  .\Objects\main.obj (MAIN)
  .\Objects\uart.obj (UART)
  C:\KEIL_V5\C51\LIB\C51S.LIB (?C_STARTUP)
  C:\KEIL_V5\C51\LIB\C51S.LIB (?C_INIT)


LINK MAP OF MODULE:  .\Objects\SN8F5835_Test Code (OPTIONS_SN8F5835)


            TYPE    BASE      LENGTH    RELOCATION   SEGMENT NAME
            -----------------------------------------------------

            * * * * * * *   D A T A   M E M O R Y   * * * * * * *
            REG     0000H     0008H     ABSOLUTE     "REG BANK 0"
            DATA    0008H     000AH     UNIT         ?DT?UART
            DATA    0012H     0001H     UNIT         ?DT?MAIN
            IDATA   0013H     0001H     UNIT         ?STACK

            * * * * * * *  X D A T A   M E M O R Y  * * * * * * *
                    0000H     F000H                  *** GAP ***
            XDATA   F000H     0001H     ABSOLUTE     
            XDATA   F001H     0001H     ABSOLUTE     
            XDATA   F002H     0001H     ABSOLUTE     
            XDATA   F003H     0001H     ABSOLUTE     
            XDATA   F004H     0001H     ABSOLUTE     
            XDATA   F005H     0001H     ABSOLUTE     
            XDATA   F006H     0001H     ABSOLUTE     
            XDATA   F007H     0001H     ABSOLUTE     
            XDATA   F008H     0001H     ABSOLUTE     
            XDATA   F009H     0001H     ABSOLUTE     
            XDATA   F00AH     0001H     ABSOLUTE     
            XDATA   F00BH     0001H     ABSOLUTE     
            XDATA   F00CH     0001H     ABSOLUTE     
            XDATA   F00DH     0001H     ABSOLUTE     
            XDATA   F00EH     0001H     ABSOLUTE     
            XDATA   F00FH     0001H     ABSOLUTE     
            XDATA   F010H     0001H     ABSOLUTE     
            XDATA   F011H     0001H     ABSOLUTE     
            XDATA   F012H     0001H     ABSOLUTE     
            XDATA   F013H     0001H     ABSOLUTE     
            XDATA   F014H     0001H     ABSOLUTE     
                    F015H     0001H                  *** GAP ***
            XDATA   F016H     0001H     ABSOLUTE     
            XDATA   F017H     0001H     ABSOLUTE     
            XDATA   F018H     0001H     ABSOLUTE     
            XDATA   F019H     0001H     ABSOLUTE     
            XDATA   F01AH     0001H     ABSOLUTE     
            XDATA   F01BH     0001H     ABSOLUTE     
BL51 BANKED LINKER/LOCATER V6.22                                                      05/19/2022  17:58:17  PAGE 2


            XDATA   F01CH     0001H     ABSOLUTE     
            XDATA   F01DH     0001H     ABSOLUTE     
            XDATA   F01EH     0001H     ABSOLUTE     
            XDATA   F01FH     0001H     ABSOLUTE     
            XDATA   F020H     0001H     ABSOLUTE     
            XDATA   F021H     0001H     ABSOLUTE     
            XDATA   F022H     0001H     ABSOLUTE     
            XDATA   F023H     0001H     ABSOLUTE     
            XDATA   F024H     0001H     ABSOLUTE     
            XDATA   F025H     0001H     ABSOLUTE     
            XDATA   F026H     0001H     ABSOLUTE     
            XDATA   F027H     0001H     ABSOLUTE     
            XDATA   F028H     0001H     ABSOLUTE     
            XDATA   F029H     0001H     ABSOLUTE     
                    F02AH     0001H                  *** GAP ***
            XDATA   F02BH     0001H     ABSOLUTE     
            XDATA   F02CH     0001H     ABSOLUTE     
            XDATA   F02DH     0001H     ABSOLUTE     
            XDATA   F02EH     0001H     ABSOLUTE     
            XDATA   F02FH     0001H     ABSOLUTE     
            XDATA   F030H     0001H     ABSOLUTE     
            XDATA   F031H     0001H     ABSOLUTE     
            XDATA   F032H     0001H     ABSOLUTE     
            XDATA   F033H     0001H     ABSOLUTE     

            * * * * * * *   C O D E   M E M O R Y   * * * * * * *
            CODE    0000H     0003H     ABSOLUTE     
            CODE    0003H     0015H     UNIT         ?PR?TIMER1_INITIALIZATION?UART
                    0018H     0003H                  *** GAP ***
            CODE    001BH     0003H     ABSOLUTE     
            CODE    001EH     008CH     UNIT         ?C_C51STARTUP
            CODE    00AAH     0060H     UNIT         ?PR?RX_RUN?UART
            CODE    010AH     005FH     UNIT         ?PR?ISR_TIMER1?UART
            CODE    0169H     0047H     UNIT         ?PR?TX_RUN?UART
            CODE    01B0H     0019H     UNIT         ?PR?MAIN?MAIN
            CODE    01C9H     0019H     UNIT         ?PR?GPIO_INITIALIZATION?MAIN
            CODE    01E2H     0019H     UNIT         ?C_INITSEG
            CODE    01FBH     0014H     UNIT         ?PR?UART_INITIALIZATION?UART
            CODE    020FH     000FH     UNIT         ?PR?_SEND_DATA?UART
                    021EH     7DD2H                  *** GAP ***
            CODE    7FF0H     0002H     ABSOLUTE     
                    7FF2H     0004H                  *** GAP ***
            CODE    7FF6H     000AH     ABSOLUTE     



OVERLAY MAP OF MODULE:   .\Objects\SN8F5835_Test Code (OPTIONS_SN8F5835)


SEGMENT
  +--> CALLED SEGMENT
---------------------
?PR?ISR_TIMER1?UART
  +--> ?PR?TX_RUN?UART
  +--> ?PR?RX_RUN?UART

?PR?RX_RUN?UART
BL51 BANKED LINKER/LOCATER V6.22                                                      05/19/2022  17:58:17  PAGE 3


  +--> ?PR?_SEND_DATA?UART

*** NEW ROOT ***************************************************

?C_C51STARTUP
  +--> ?PR?MAIN?MAIN
  +--> ?C_INITSEG

?PR?MAIN?MAIN
  +--> ?PR?GPIO_INITIALIZATION?MAIN
  +--> ?PR?TIMER1_INITIALIZATION?UART
  +--> ?PR?UART_INITIALIZATION?UART
  +--> ?PR?_SEND_DATA?UART



SYMBOL TABLE OF MODULE:  .\Objects\SN8F5835_Test Code (OPTIONS_SN8F5835)

  VALUE           TYPE          NAME
  ----------------------------------

  -------         MODULE        OPTIONS_SN8F5835
  C:7FF0H         PUBLIC        CRC_CHECK_DATA
  N:001EH         SYMBOL        BIT16_BYPASS1P_H
  N:00AFH         SYMBOL        BIT16_BYPASS1P_L
  N:0008H         SYMBOL        CK_FINE_TUNING_SET
  N:0018H         SYMBOL        CLOCKSRC_SET
  N:00C0H         SYMBOL        EXTERNAL_CLOCKRATE_SET
  N:00A0H         SYMBOL        IHRC32M_CLOCKRATE_SET
  N:0004H         SYMBOL        ISP_EN_SET
  N:0001H         SYMBOL        NOISEFILT_SET
  N:0030H         SYMBOL        RESETPIN_SET
  N:8000H         SYMBOL        ROM_SIZE
  N:0003H         SYMBOL        SECURITY_SET
  N:00C0H         SYMBOL        WATCHCLK_SET
  N:00A0H         SYMBOL        WATCHDOG_SET
  N:00C0H         SYMBOL        XTAL12M_CLOCKRATE_SET
  N:00E0H         SYMBOL        XTAL4M_CLOCKRATE_SET
  -------         ENDMOD        OPTIONS_SN8F5835

  -------         MODULE        MAIN
  C:0000H         SYMBOL        _ICE_DUMMY_
  X:F003H         PUBLIC        PW1YL
  X:F017H         PUBLIC        PW2YL
  D:0080H         PUBLIC        P0
  X:F031H         PUBLIC        PW3YL
  D:0090H         PUBLIC        P1
  D:00B0H         PUBLIC        P3
  D:00C8H         PUBLIC        P4
  D:00A0H         PUBLIC        TTCON
  D:00A8H         PUBLIC        IEN0
  D:00B8H         PUBLIC        IEN1
  D:0012H         PUBLIC        UART_Model
  X:F004H         PUBLIC        PW10DH
  X:F018H         PUBLIC        PW20DH
  X:F006H         PUBLIC        PW11DH
  X:F01AH         PUBLIC        PW21DH
BL51 BANKED LINKER/LOCATER V6.22                                                      05/19/2022  17:58:17  PAGE 4


  X:F00CH         PUBLIC        PW30DH
  X:F008H         PUBLIC        PW12DH
  X:F01CH         PUBLIC        PW22DH
  X:F00EH         PUBLIC        PW31DH
  X:F00AH         PUBLIC        PW13DH
  X:F01EH         PUBLIC        PW23DH
  X:F010H         PUBLIC        PW32DH
  X:F005H         PUBLIC        PW10DL
  X:F019H         PUBLIC        PW20DL
  X:F012H         PUBLIC        PW33DH
  X:F007H         PUBLIC        PW11DL
  X:F01BH         PUBLIC        PW21DL
  X:F00DH         PUBLIC        PW30DL
  X:F009H         PUBLIC        PW12DL
  X:F01DH         PUBLIC        PW22DL
  X:F00FH         PUBLIC        PW31DL
  X:F00BH         PUBLIC        PW13DL
  X:F01FH         PUBLIC        PW23DL
  X:F011H         PUBLIC        PW32DL
  X:F013H         PUBLIC        PW33DL
  X:F000H         PUBLIC        PW1M
  C:01B0H         PUBLIC        main
  X:F014H         PUBLIC        PW2M
  X:F02DH         PUBLIC        HIDR
  X:F028H         PUBLIC        P0UR
  X:F001H         PUBLIC        PW3M
  X:F029H         PUBLIC        P1UR
  X:F02BH         PUBLIC        P3UR
  X:F02CH         PUBLIC        P4UR
  D:00D8H         PUBLIC        CSCON4
  D:0088H         PUBLIC        TCON
  X:F027H         PUBLIC        TSWA
  X:F026H         PUBLIC        TSWB
  D:0086H         PUBLIC        WDTR
  X:F025H         PUBLIC        TSWD
  D:00F9H         PUBLIC        P0M
  D:00FAH         PUBLIC        P1M
  D:00FBH         PUBLIC        P3M
  D:00FCH         PUBLIC        P4M
  X:F02EH         PUBLIC        CSADB1H
  X:F024H         PUBLIC        TSWY
  X:F032H         PUBLIC        CSADB2H
  X:F02FH         PUBLIC        CSADB1L
  X:F033H         PUBLIC        CSADB2L
  C:01C9H         PUBLIC        GPIO_Initialization
  D:0098H         PUBLIC        S0CON
  X:F022H         PUBLIC        MINCS0H
  X:F020H         PUBLIC        MAXCS0H
  X:F023H         PUBLIC        MINCS0L
  X:F021H         PUBLIC        MAXCS0L
  X:F002H         PUBLIC        PW1YH
  D:00D0H         PUBLIC        PSW
  X:F016H         PUBLIC        PW2YH
  X:F030H         PUBLIC        PW3YH
  D:00C0H         PUBLIC        IRCON
  -------         PROC          MAIN
  C:01B0H         LINE#         34
BL51 BANKED LINKER/LOCATER V6.22                                                      05/19/2022  17:58:17  PAGE 5


  C:01B0H         LINE#         35
  C:01B0H         LINE#         36
  C:01B3H         LINE#         37
  C:01B6H         LINE#         38
  C:01B9H         LINE#         39
  C:01BCH         LINE#         40
  C:01BFH         LINE#         41
  C:01BFH         LINE#         42
  C:01BFH         LINE#         43
  C:01C2H         LINE#         44
  C:01C7H         LINE#         45
  -------         ENDPROC       MAIN
  -------         PROC          GPIO_INITIALIZATION
  C:01C9H         LINE#         49
  C:01C9H         LINE#         50
  C:01C9H         LINE#         52
  C:01CFH         LINE#         53
  C:01D5H         LINE#         54
  C:01DBH         LINE#         55
  C:01E1H         LINE#         56
  -------         ENDPROC       GPIO_INITIALIZATION
  -------         ENDMOD        MAIN

  -------         MODULE        UART
  C:0000H         SYMBOL        _ICE_DUMMY_
  D:0080H         PUBLIC        P0
  D:0090H         PUBLIC        P1
  D:00B0H         PUBLIC        P3
  D:00C8H         PUBLIC        P4
  C:010AH         PUBLIC        ISR_Timer1
  C:020FH         PUBLIC        _Send_data
  D:00A0H         PUBLIC        TTCON
  D:00A8H         PUBLIC        IEN0
  D:00B8H         PUBLIC        IEN1
  D:0008H         PUBLIC        bRead_num_count
  D:00D8H         PUBLIC        CSCON4
  D:0009H         PUBLIC        bSend_num_count
  B:0080H.0       PUBLIC        P00
  B:0080H.1       PUBLIC        P01
  B:0080H.2       PUBLIC        P02
  D:0089H         PUBLIC        TMOD
  D:0088H         PUBLIC        TCON
  D:000AH         PUBLIC        bRead_buffer
  D:000BH         PUBLIC        bSend_buffer
  D:00F9H         PUBLIC        P0M
  D:008DH         PUBLIC        TH1
  D:008BH         PUBLIC        TL1
  B:00A8H.7       PUBLIC        EAL
  D:000CH         PUBLIC        bRead_flag
  D:000DH         PUBLIC        bRead_data
  C:00AAH         PUBLIC        RX_run
  C:0169H         PUBLIC        TX_run
  D:0098H         PUBLIC        S0CON
  D:00E7H         PUBLIC        TCON0
  C:0003H         PUBLIC        TIMER1_Initialization
  D:000EH         PUBLIC        bSend_flag
  D:000FH         PUBLIC        bSend_data
BL51 BANKED LINKER/LOCATER V6.22                                                      05/19/2022  17:58:17  PAGE 6


  D:0010H         PUBLIC        bRead_count
  C:01FBH         PUBLIC        UART_Initialization
  D:00D0H         PUBLIC        PSW
  D:0011H         PUBLIC        bSend_count
  D:00C0H         PUBLIC        IRCON
  -------         PROC          TIMER1_INITIALIZATION
  C:0003H         LINE#         29
  C:0003H         LINE#         31
  C:0003H         LINE#         38
  C:0006H         LINE#         39
  C:0009H         LINE#         40
  C:000CH         LINE#         41
  C:000FH         LINE#         42
  C:0012H         LINE#         43
  C:0014H         LINE#         44
  C:0017H         LINE#         47
  -------         ENDPROC       TIMER1_INITIALIZATION
  -------         PROC          UART_INITIALIZATION
  C:01FBH         LINE#         48
  C:01FBH         LINE#         49
  C:01FBH         LINE#         50
  C:0205H         LINE#         51
  C:020EH         LINE#         52
  -------         ENDPROC       UART_INITIALIZATION
  -------         PROC          ISR_TIMER1
  C:010AH         LINE#         53
  C:0127H         LINE#         61
  C:012AH         LINE#         62
  C:012DH         LINE#         63
  C:0130H         LINE#         64
  C:0133H         LINE#         65
  C:0137H         LINE#         66
  C:0137H         LINE#         67
  C:013AH         LINE#         68
  C:013CH         LINE#         69
  C:0141H         LINE#         70
  C:0141H         LINE#         71
  C:0141H         LINE#         72
  C:0143H         LINE#         73
  C:0148H         LINE#         74
  C:0148H         LINE#         75
  C:014BH         LINE#         76
  C:014EH         LINE#         77
  C:014EH         LINE#         79
  -------         ENDPROC       ISR_TIMER1
  -------         PROC          _SEND_DATA
  D:0007H         SYMBOL        output
  C:020FH         LINE#         86
  C:020FH         LINE#         87
  C:020FH         LINE#         88
  C:0213H         LINE#         89
  C:0213H         LINE#         90
  C:0215H         LINE#         91
  C:0218H         LINE#         92
  C:021BH         LINE#         93
  C:021BH         LINE#         95
  C:021BH         LINE#         96
BL51 BANKED LINKER/LOCATER V6.22                                                      05/19/2022  17:58:17  PAGE 7


  C:021DH         LINE#         97
  C:021DH         LINE#         98
  -------         ENDPROC       _SEND_DATA
  -------         PROC          TX_RUN
  C:0169H         LINE#         99
  C:0169H         LINE#         100
  C:0169H         LINE#         109
  C:016BH         LINE#         110
  C:0170H         LINE#         111
  C:0170H         LINE#         112
  C:0172H         LINE#         113
  C:0175H         LINE#         114
  C:0178H         LINE#         115
  C:0178H         LINE#         116
  C:0184H         LINE#         117
  C:0184H         LINE#         118
  C:0186H         LINE#         119
  C:018DH         LINE#         120
  C:018DH         LINE#         121
  C:0190H         LINE#         122
  C:0195H         LINE#         123
  C:0195H         LINE#         124
  C:0197H         LINE#         125
  C:0199H         LINE#         127
  C:0199H         LINE#         128
  C:019BH         LINE#         129
  C:019BH         LINE#         130
  C:01A1H         LINE#         132
  C:01A2H         LINE#         133
  C:01A7H         LINE#         134
  C:01A7H         LINE#         135
  C:01A9H         LINE#         136
  C:01AAH         LINE#         138
  C:01AAH         LINE#         139
  C:01ADH         LINE#         140
  C:01AFH         LINE#         141
  C:01AFH         LINE#         142
  C:01AFH         LINE#         143
  -------         ENDPROC       TX_RUN
  -------         PROC          RX_RUN
  C:00AAH         LINE#         144
  C:00AAH         LINE#         145
  C:00AAH         LINE#         152
  C:00ACH         LINE#         153
  C:00B3H         LINE#         154
  C:00B3H         LINE#         155
  C:00B6H         LINE#         156
  C:00B8H         LINE#         157
  C:00B8H         LINE#         158
  C:00C2H         LINE#         159
  C:00C2H         LINE#         160
  C:00C5H         LINE#         161
  C:00C8H         LINE#         162
  C:00C8H         LINE#         163
  C:00D4H         LINE#         164
  C:00D4H         LINE#         165
  C:00D6H         LINE#         166
BL51 BANKED LINKER/LOCATER V6.22                                                      05/19/2022  17:58:17  PAGE 8


  C:00DDH         LINE#         167
  C:00DDH         LINE#         168
  C:00E3H         LINE#         169
  C:00E6H         LINE#         170
  C:00E6H         LINE#         171
  C:00EAH         LINE#         172
  C:00EAH         LINE#         173
  C:00EBH         LINE#         175
  C:00EBH         LINE#         176
  C:00EEH         LINE#         177
  C:00F0H         LINE#         180
  C:00F5H         LINE#         181
  C:00F8H         LINE#         182
  C:00FDH         LINE#         183
  C:0100H         LINE#         185
  C:0100H         LINE#         186
  C:0101H         LINE#         187
  C:0106H         LINE#         188
  C:0106H         LINE#         189
  C:0109H         LINE#         190
  C:0109H         LINE#         191
  -------         ENDPROC       RX_RUN
  -------         ENDMOD        UART

Program Size: data=20.0 xdata=50 code=551
LINK/LOCATE RUN COMPLETE.  0 WARNING(S),  0 ERROR(S)
